:1000000002308A00692A0000FF30831685008600CE
:100010008312061583160611831286148316861022
:100020008312051583160511831285158316851114
:100030008312051683160512831206148316061002
:1000400083128615831686118312861683168612EE
:1000500083120616831606128312861783168613DA
:1000600083120510831605108730831290008A11C1
:10007000722A2908013A03194128033A031945282D
:100080004928861C861406114A28061D0615861066
:100090004A284A2808002908013A03195928033A2E
:1000A00003196128063A031969280C3A03197128C3
:1000B0007928851D8515051E0516061C06140511D3
:1000C0007A28051D0515051E0516061C0614851142
:1000D0007A28851D8515051D0515061C06140512B3
:1000E0007A28851D8515051E0516051D05150610A2
:1000F0007A287A2808002808013A03199528033A33
:1001000003199C28013A0319A328073A0319AA28BE
:10011000013A0319B128033A0319B828013A03191F
:10012000BF280F3A0319C628CD280130A90039206D
:100130000830A9004B20CE280230A9003920083011
:10014000A9004B20CE280130A90039200430A90095
:100150004B20CE280230A90039200430A9004B20C2
:10016000CE280130A90039200230A9004B20CE282A
:100170000230A90039200230A9004B20CE280130DE
:10018000A90039200130A9004B20CE280230A90057
:1001900039200130A9004B20CE28CE2808002B3072
:1001A0008400831300080319E3280330F800F701E3
:1001B000F70BD828F80BD7283C30F700F70BDE28D0
:1001C000E128800BD5280800861586128F018E0144
:1001D0000130AB00CF200F08FA000E08F7000F081F
:1001E0007A02031DEB287708A8007A08A900A9085D
:1001F000031DFE282808293C03180829A908031D07
:10020000082928082D3C031C08290130AA008C2944
:10021000A908031D0F2928082D3C03181929A9082E
:10022000031D19292808323C031C19290230AA0091
:100230008C29A908031D20292808553C03182A29C0
:10024000A908031D2A2928085A3C031C2A2903301F
:10025000AA008C29A908031D312928085D3C031830
:100260003B29A908031D3B292808623C031C3B29A4
:100270000430AA008C29A908031D42292808A93C9A
:1002800003184C29A908031D4C292808B43C031C59
:100290004C290530AA008C29A908031D53292808D8
:1002A000B83C03185D29A908031D5D292808C83C2E
:1002B000031C5D290630AA008C292908003C03187C
:1002C0007529FF3A031D68292808583C0318752929
:1002D0002908013C031C7529031D722928086D3C5F
:1002E000031C75290730AA008C292908003C031833
:1002F0008C29FF3A031D80292808763C03188C2995
:100300002908013C031C8C29031D8A2928088B3CE1
:10031000031C8C290830AA002A08AB002B08013ADC
:100320000319A829033A0319AC29013A0319B02982
:10033000073A0319B429013A0319B829033A0319F2
:10034000BC29013A0319C0290F3A0319C429C82945
:10035000A1012830A000C929A1012830A000C92985
:10036000A1012830A000C929A1012830A000C92975
:10037000A1015D30A000C929A1015530A000C92903
:10038000A1012E30A000C929A1012A30A000C9294D
:10039000C9292A08F8008A117A2A861686118F013F
:1003A0008E010130AB00CF200F08FA000E08F700D5
:1003B0000F087A02031DD4297708A9007A08AA0039
:1003C000A808031DE6290030F800672A2808013A2A
:1003D0000319002A033A03190B2A013A0319162AB2
:1003E000073A0319212A013A03192C2A033A03195F
:1003F0003A2A013A0319482A0F3A0319562A642A5D
:10040000AA08031D0A2A2908593C031C0A2A00309D
:10041000F800672A652AAA08031D152A2908633CE3
:10042000031C152A0030F800672A652AAA08031D54
:10043000202A2908BD3C031C202A0030F800672A26
:10044000652AAA08031D2B2A2908D13C031C2B2A44
:100450000030F800672A652A2A08013C031C392A63
:10046000031D362A29087B3C031C392A0030F8007A
:10047000672A652A2A08013C031C472A031D442ACF
:100480002908A33C031C472A0030F800672A652A84
:100490002A08033C031C552A031D522A29081F3C25
:1004A000031C552A0030F800672A652A2A08033CF5
:1004B000031C632A031D602A2908833C031C632A4A
:1004C0000030F800672A652A652A0130F8008A1191
:1004D0007F2A840183131F308305073083169C0015
:1004E000831204280130A8007B20A401A501A701E4
:1004F000A601E4287808A2002208A800CD297808DF
:10050000A300240822020319942AA2080319942A9A
:100510002208A4002208A400A8007B200616861743
:100520000510A501A701A601A308031D9E2A061612
:1005300086170510A501A701A601A42AA208031980
:10054000A42A06120130A500A5080319B72A21081C
:100550002702031CB42A031DB12A2608200203180F
:10056000B42A05148613B72AA60A0319A70A792AFA
:02057000630026
:04400E00021FFF3F4F
:00000001FF
